:10000000E7280530AC00A530AD00AD0B0528AC0BE2
:10001000032800348600003066000515851005149D
:100020000510FF3066000511851405140608AF00A1
:10003000AF1705100514861F1F2805101A28051074
:100040003228860000306600051185100514051061
:10005000FF30660085140514861F302805102B28F4
:10006000051000342F1C0034AF1C00342F1D003449
:10007000AF1D00343930AF07AF172F082128831385
:1000800010088D0203184B2801308E0203184B28EC
:100090008F02031C831711088E02031853280130A6
:1000A0008F02031C831712088F02031C831700346E
:1000B00010088D07031C5F288E0F5F288F0A110818
:1000C0008E0703188F0A12088F0700340730AC0020
:1000D000193084002F308000840AAC0B6B280F305D
:1000E000920042309100403090003F20990A3A300F
:1000F00019060319EB29831F752858200130920037
:1001000086309100A03090003F209A0A831F8428F7
:100110005820920127309100103090003F209B0A18
:10012000831F8E28582003309100E83090003F2034
:100130009C0A831F972858209101643090003F202B
:100140009D0A831F9F2858200A3090003F209E0A56
:10015000831FA62858200D089F079F0A00343730B8
:10016000620010306500851105118F018101960133
:10017000051505110C08AC008515FA30AD00C62830
:1001800000000000000000000000000001089602CE
:10019000031DCC280000CE2803188F0A960000000B
:1001A00000000000AD0BC028AC0BBD288511010874
:1001B0008E009602031CDE28031D8F0A8D018D031D
:1001C0000515051101080E060319DF280034850105
:1001D00010306500860100306600012001200120FA
:1001E0003830860005140120051005140120051083
:1001F000051401200510383021200C302120013059
:1002000021200630212014308C00AF2066203030B1
:100210001906031D0F2930301A0603194E298230A2
:1002200021200230AC001930840030300006031D5C
:100230001F2920300A20840AAC0B15292429000824
:100240000A20840AAC0B1F292E300A200530AC008E
:1002500000080A20840AAC0B282920300A204D30DF
:100260000A2048300A207A300A2020300A20203024
:100270000A20032914308C00AF2066203030190684
:10028000031D0F2932301A0203180F2930301A06C5
:10029000031D4E2930301B06031977298230212097
:1002A0000530AC001930840030300006031D5E2993
:1002B00020300A20840AAC0B5429632900080A2044
:1002C000840AAC0B5E292E300A2000080A20840A1A
:1002D00000080A2020300A204B300A2048300A202B
:1002E0007A300A2020300A2020300A203A29C830EB
:1002F0008C00AF20662030301906031D3A293230B9
:100300001A0203183A2930301A06031D8B2930309F
:100310001B060319C729823021200430AC00193094
:10032000840030300006031D9B2920300A20840AF7
:10033000AC0B9129A02900080A20840AAC0B9B2948
:100340002E300A2000080A20840A00080A20840AA5
:1003500000080A2020300A204B300A2048300A20AA
:100360007A300A2020300A2020300A207729C8302D
:100370008C00AF20662030301906031D8B293030E9
:100380001A06031D8B2932301B0203188B29823079
:1003900021200730AC001930840030300006031DE6
:1003A000D72920300A20840AAC0BCD29DC2900088B
:1003B0000A20840AAC0BD72920300A2048300A20B2
:1003C0007A300A2020300A2020300A2020300A20EB
:1003D00020300A20B72901302120843021204F30DD
:1003E0000A2076300A2065300A2072300A206630F2
:1003F0000A206C300A206F300A2077300A20023041
:04040000212003298B
:00000001FF
